:104A1E00C10CC1094113410042133F000041134331
:0E4A2E00014113060144130CFFFFFFFFC10BF3
:10345400EFFD3395E0FC740C2DF58274133CF58379
:10346400222582F582E43583F5837401F09013F10B
:10347400E475F0010214C79011CA12180789828AF0
:103484008322EEFD3395E0FC74072DF58274133C22
:10349400F58322900FB6E0D36480F8EE648098221E
:1034A4009013F2E025E0FF9013F1E033FE74162F41
:1034B400F58274053EF583229013F1E0FEA3E0FF4C
:1034C40022E49013F1F0A3F02290133EE0FF901455
:1034D4004BE06F22EDFF3395E0FEEF25E0FFEE3386
:1034E400FE2274FC2FF58274053EF58322FBEAC4A8
:1034F400F854F0C8EBC4540F4890149BF022901376
:10350400F1E0FCA3E02224DEF58274053EF583E0BD
:1035140022125A58900FB9E0223EF583EAF0A3EB49
:10352400F0223EF583E0FAA3E02225E02480F58230
:10353400E43405F5832290144CE0FFA3E0FDA3E0FE
:10354400FB22EC25E02425F8E6FA08E6229FEE6447
:0735540080F8E0648098227A
:105A6F0075840F75A4357580C075A57C75A7FF75F6
:065A7F00E11775E344226B
:0F5BAC00E4F584759A4075F809759D01C2FA22D7
:1056F500E4F584758850758921F58E758DEB75C92E
:105705000875CDFF75CCC075CBFF75CAE075C804AB
:03571500F58422F6
:105B7A00E4F584759105759852758401F598F58454
:015B8A0022F8
:104F7000E4FFFE75840F438A0353A1DFF58475B700
:104F80003075840F43A120438901758D01758F0110
:104F9000758E040FBF00010EEF640F4E70F543894C
:104FA00002E58920E4130FBF00010EBE0FF3BFFF1F
:0C4FB000F0E4F58443EF1080E8759702F0
:014FBC0022D2
:0A5C3B0075A89275B81075E60822EE
:105B5600E4F58475D84075D98375DA3175DB31D2B1
:025B6600DE223D
:105AB100125A6F124F701256F5125B56125B7A1220
:055AC1005BAC025C3B40
:105B1A007F01125A587F03125A587F011259DA7FAD
:045B2A00030259DA3F
:105B2E007F021259DA7F041259DA7F02125A587F15
:045B3E0004025A58AB
:023B4900AC07C7
:103B4B00E490149CF0ED443090149AF0E4FD746111
:103B5B002DF8E66C705790149C04F01234D87495C1
:103B6B002FF58274021235261234F1EB540FF91231
:103B7B0034D874D92FF5827401123526FB74952F26
:103B8B00F582740212351D74F02FF5827400123514
:103B9B0026FB74D92FF582740112351D123546FBA5
:103BAB001234D874F02FF582740012351D0DED64AC
:103BBB0004709B90149CE0700C1235461234F1AFDC
:103BCB0003EF540FF9E9C454F0F9E59A20E7FBE44D
:103BDB00F59BE59A20E7FB90149AE0F59BE59A207C
:103BEB00E7FB90149BE0F59BE59A20E7FB899BE5AF
:0B3BFB009A20E7FBAF05EF3395E0FEDA
:013C0600229B
:053F5D009014A6EFF036
:103F620012185C3F81003F8E013F9B023FA8033F36
:103F7200B5043FC2053FCF063FDC0700003FE77FA5
:103F8200061218919014A77405F080597F06122525
:103F9200DB9014A77406F0804C7F0612442790141D
:103FA200A77407F0803F7F06123A869014A7740820
:103FB200F080327F071218919014A77409F08025BF
:103FC2007F071225DB9014A7740AF080187F07126E
:103FD20044279014A7740BF0800B7F07123A869047
:103FE20014A7740CF0D282C2959014A7E0FF90142B
:0A3FF200A6E0FD123B49D295C28201
:013FFC0022A2
:053FFD009014A8EFF094
:1040020012185C402100402E01403B024048034010
:104012005504406205406F06407C07000040877FE0
:10402200081218919014A9740DF080597F08122576
:10403200DB9014A97412F0804C7F0812442790146C
:10404200A9740FF0803F7F08123A869014A9741069
:10405200F080327F091218919014A97411F0802512
:104062007F091225DB9014A9740EF080187F0912C3
:1040720044279014A97413F0800B7F09123A86909A
:1040820014A97414F0D282C2969014A9E0FF90147D
:0A409200A8E0FD123B49D296C2825D
:01409C002201
:054DD2009014AAEFF0AF
:104DD70024FA601704702B9014AB741DF09013C560
:104DE7007403F07B277D2A7F1D80129014AB741CFF
:104DF700F09013C57402F07B117D1F7F1C1233499D
:104E0700800A9014AAE0FFA3F0122360D282C29412
:104E17009014ABE0FF9014AAE0FD123B49D294C274
:014E27008208
:014E28002267
:054D7A009014ACEFF005
:104D7F0024FA601704702A9014AD741BF09013C5B9
:104D8F007401F07B287D2B7F1B80119014AD741A5A
:104D9F00F0E49013C5F07B127D207F1A1233498007
:104DAF000C9014ACE02415FFA3F01241D2D282C2B2
:104DBF00979014ADE0FF9014ACE0FD123B49D297F1
:024DCF00C2829E
:014DD10022BF
:0F5BBB009013057407F0D294D295D296D2972208
:10355B009014AEE584F0A3E5A8F09011B112180712
:10356B00E94A700302365853A87DE4F58453F87F7B
:10357B00901344F0A3F0C2B3901267E0FFB40118AC
:10358B0090119BE0C313FE7402A806088002C3339C
:10359B00D8FC901344F0806CEFB40216901239E013
:1035AB00FF7401A807088002C333D8FC901345F0C1
:1035BB008052901267E0B4034B9011A0E012185C9C
:1035CB0035ED0035ED0135F50235F50335FD0435E7
:1035DB00FD05360506360507360D08360D090000C4
:1035EB00360F9013457410F0801A9013457420F029
:1035FB0080129013457440F0800A9013457480F04C
:10360B008002D2B3300A07901344E04440F0C2FA70
:10361B00E4FF0FEFB432FB53F87FE59A20E7FB9002
:10362B001344E0F59BE4FF0FEFB432FB53F87FE557
:10363B009A20E7FB901345E0F59BE4FF0FEFB432C4
:0D364B00FBD2FA9014AEE0F584A3E0F5A8E0
:01365800224F
:031A0600023E1687
:103E1600C0E0C0F0C083C082C0D075D000C000C072
:0D3E260001C002C003C004C005C006C007F3
:103E330090133F123474901305E014F0E0C3940719
:103E430050037426F0901305E0FF131313541FFE61
:103E5300EF54079014C8F0AF06EF24FE6018146007
:103E63001F1460262403702E9014C8E0FF640760BB
:103E730025124DD280209014C8E0FF123F5D8016BA
:103E83009014C8E0FF123FFD800C9014C8E0FF645B
:0C3E9300076003124D7A758AFF758CFFE2
:103E9F00D007D006D005D004D003D002D001D00077
:0B3EAF00D0D0D082D083D0F0D0E03221
:0A5C4500EF12352EECF0A3EDF02273
:1054E50090134CE0FEA3E0FF901348E0FCA3E0FD21
:1054F500B50719ECB50615901351E0FEA3E0FFEDD5
:0E550500B50709ECB5060520C502D322C32266
:1049B500E4FE1234975011EE123455E0F4600612FD
:1049C500348CE004F00E80EA901310E0123455EFB9
:1049D500F012348CE4F0FE1234975011EE12345577
:1049E500E0B4FF06901310EEF0220E80EAE4901377
:1049F50010F0901307E0FF7E01123497501A12341D
:104A050086E0FDD3EF6480F8ED6480984007AF053C
:084A1500901310EEF00E80E199
:014A1D002276
:053C07009014B0EFF085
:103C0C00E4FF900FB6E0D36480F8EF648098506BBB
:103C1C00123454E0FE9014B0E0FDEE6D7059123485
:103C2C005474FFF012348C74FFF09014B1747FF064
:103C3C00E4FE123497501CEE6F6015123486E0FDD2
:103C4C009014B1E0C36480F8ED6480985002EDF0FC
:103C5C000E80DFE4FE1234975021EE6F60161234A2
:103C6C0086C083C082E0FD9014B1E0FCC3ED9CD013
:103C7C0082D083F00E80DE0F023C0EE4901310F025
:103C8C00FF900FB6E0FED36480F8EF64809850107C
:103C9C00123454E0F4601A901310E004F00F80E139
:103CAC00EE14FF901310E0FED3EF12349C4002EFA1
:013CBC00F017
:013CBD0022E4
:1059DA007584014398028F99E59870047F018002CB
:0A59EA007F00EF20E1F2E4F58422D3
:105A5800E4F5844398028F99E59870047F018002E9
:075A68007F00EF20E1F222B4
:024CC600A9073C
:104CC800E49014B2F0A3F0E9FF3395E0FEC390142A
:104CD800B3E09014B2123551503EE4FFFEE9FD33C3
:104CE80095E0FCC3EF9DEC12349C5024E4FDFCE9F4
:104CF800FB3395E0FAC3ED9BEA6480F8EC64809896
:104D080050070DBD00010C80E60FBF00010E80CDDD
:084D18009014B212347480AF54
:014D20002270
:100C9A00E4900FB6F0FBFAF99011B112182775FF1C
:100CAA00DE75FFADE4F5E6F5E7125A27125AB112DE
:100CBA0052771259F4125BBB12575E125B8BE4F542
:100CCA008475D48475D48475D10375D340D28112C6
:100CDA00589FD2AFD2FF1234C590133E7440F0E44D
:100CEA00901310F01234C6900FB6E0FF3395E0FE71
:100CFA00D39013F2E09013F11235515022E0FEA383
:100D0A00E0FF240CF58274133EF58374FFF0740738
:100D1A002FF58274133EF58374FF12347080C8E491
:100D2A001213831245451258BD125C4F12355B7F70
:100D3A0039125A58C209125B687E00EF64016003D7
:100D4A000211B9125862EF64B060030211B990132C
:100D5A00F9F01234C61234BCC3942DEE6480948028
:100D6A00501474112FF58274133EF583E4F0901336
:100D7A00F112347580DF1234C51234BCC3941BEEF1
:100D8A00648094805028123502FD24FCF582740593
:100D9A003CF583E0FB74DE2DF58274053CF583EBAC
:100DAA00F01234E6E4F09013F112347580CBC218D5
:100DBA00125B68EF60FA1258629013F3EFF05480F6
:100DCA00FFE4FCFDFEEF7003020F31E0FF64C07028
:100DDA0003020F31EF64B07003020F319013F9E090
:100DEA0004F09013F3E0547FFF9013F5F07419D3D5
:100DFA009F500DE0FF94265007EF24F2A3F0802ABB
:100E0A009013F5E0FFE4D39F500AEF94185005A31E
:100E1A00EFF08016EFB429089013F67419F0800ADF
:100E2A00EFB42C069013F6741AF09013F6E0FFC391
:100E3A00941B500D74FC2FF582E43405F58374017C
:100E4A00F0E49013F7F0A3F0125B68EF60FA12581F
:100E5A00629013F4EFF0125B68EF60FA125862AD19
:100E6A00079013F4E0FF9013F7E0F0A3E04FF0903F
:100E7A0013F7E0FEA3E07806C333CE33CED8F9F0F9
:100E8A00EE9013F7F0AF05E0F0A3E04FF09013F502
:100E9A00E012352EE0FEA3E04E705E1234C6123424
:100EAA00BCC39405EE64809480501FEF75F02DA4A6
:100EBA0024F8F582E43400F583C083C0829013F5E8
:100ECA00E0D082D08312346580D41234C51234BC87
:100EDA00C39404EE64809480501FEF75F02DA4240F
:100EEA00E1F582E43401F583C083C0829013F5E012
:100EFA00D082D08312346580D49013F5E0FF90132A
:100F0A00F7E0FCA3E0FD125C459013F5E0FF241125
:100F1A00F582E43413F5837401F090130BEFF0209B
:100F2A0018051256D1D2189013F3E064C060030278
:100F3A000DBA901238E06008124BAB300C02C20CAA
:100F4A001234C51234BCC3941BEE648094804003EF
:100F5A000210DC74DE2F12350C600302108E90131F
:100F6A00F1A3E024FC1234E9E06401600302108E6C
:100F7A009013FAF0A3F09013FAE0FEA3E0FFC394F3
:100F8A0004EE64809480504C900DC275F07DEF128F
:100F9A0017E2EE75F07DA42583F583C083C0821223
:100FAA0034BCD082D08375F0051217E2EE75F005D5
:100FBA00A42583F583E0540F60129013FAE0FCA392
:100FCA00E024DAF58274053CF583EFF09013FA1207
:100FDA00347480A29013F1A3E0FF1249B5123502CE
:100FEA00FD25E0FFEC1234AF7414F0A3E4F074961C
:100FFA002FF58274003EF583C083C082E04410FF5F
:10100A00A3E0D082D083CFF0A3EFF0901238E07043
:10101A00030210D6ED64124C60047F0180027F0047
:10102A00123502FD64114C60047E0180027E00EEDE
:10103A005F70030210D6D20C9011AE1218078D827F
:10104A008C8374051217D11213A7540F70047F01F1
:10105A0080027F00EF540FFF9011AE12180712356D
:10106A0002F5828C8374051217D1E92582F9EA35D3
:10107A0083FA12138E54F04F1213F6121A1B125CD3
:01108A004F16
:10108B000210D61234BC12350AB4010B1234E6E04E
:10109B007005123C0780341234BC12350A6401709F
:1010AB002A1234E6E0B401231234A4E0FCA3E0D30B
:1010BB009400EC9402400D1234B174FE75F00012E2
:1010CB0014C780071234A4E4F0A3F0123471020F9A
:1010DB004D1234C5FDFC900615E0FF601C9005F722
:1010EB00E070160D900FB8E090130660057401F0D8
:1010FB008007E0FEC374019EF0EF70159005F7E0DA
:10110B00600F7C007D01900FB8E06005E490130642
:10111B00F0900616E0FF60229005F8E0701C90132B
:10112B00F1F0A304F0900FB7E09013436005740146
:10113B00F08007E0FEC374019EF0EF70199005F884
:10114B00E060139013F1E4F0A304F0900FB7E060AC
:10115B0005E4901343F09013F1E07002A3E06025D7
:10116B00901343E0600F7F0212351560047F0480FB
:10117B00117F02800D7F0112351560047F03800201
:10118B007F011259DAED4C6025901306E0600F7F5A
:10119B000412351560047F0280117F04800D7F03DC
:1011AB0012351560047F0180027F031259DA125643
:1011BB0037EF7003021269124ED4EF12185C12341F
:1011CB0001122902123F0411F50511EE0612030755
:1011DB0011FC08121109120A0A121F0B12180C002B
:1011EB0000125312347B7FFF802F12347B7F0180E0
:1011FB002812347B7FFE802112347B7F02801A12EF
:10120B00347B7FFD801312347B7F03800C12347B85
:10121B007FFC800512347B7F041218868027901286
:10122B006C121807121882801C9011CD121807121D
:10123B0018828011300B04B20A800AE4900D48F03A
:10124B00125A40C20A12355B125637EF6003021175
:10125B00C290133F7427F0A37410F0125C4F12541A
:10126B00B5EF7003020D3E300A2190144AE0146072
:10127B000F04701790144BE0121383125C4F800B0A
:10128B0090144BE0900D48F0125A4090144AE0FF36
:10129B00B40B02D20BEF6431701E1234CD701912E5
:1012AB0054E550FB121366A3E09013D7F012382AC3
:1012BB001254E550FB12137A90144AE06432701802
:1012CB001234CD70131254E550FB1213661238F71B
:1012DB001254E550FB12137A90144AE0642D702AD5
:1012EB001234CD70251254E550FB90133EE0FF12E3
:1012FB005AF01254E550FB12353A1241391254E5AB
:10130B0050FB90133EE0FF125ADB90144AE0642E20
:10131B00702A1234CD70251254E550FB90133EE029
:10132B00FF125AF01254E550FB12353A12426A1270
:10133B0054E550FB90133EE0FF125ADB90144AE049
:10134B00B41405D20A12355B90144AE0641560039D
:0B135B00020D3EC20A12355B020D3E7F
:1013660090133EE0FF125AF090144CE0FFA3E0FD0C
:10137600A3E0FB2290133EE0FF125ADB22900D48B9
:08138600F0125594125B2E22B7
:064A3C00046105090D11E3
:101D86003EF583ECF0A3EDF0C3ED9BFDEC9AFCE988
:101D9600FF3395E0FEEF25E0FFEE33FE22ED75F012
:101DA6002DA424F8F582E43400F583E5822EF5822D
:101DB600E43583F58322E025E0249CF582E43405AE
:101DC600F583E0FCA3E0FDEF25E02480F582E43412
:101DD60005F583E0FEA3E0229005F912182790147A
:101DE6009DE0900D4AFF75F0040217E2E09005F9B8
:101DF60075F07DA424C2F9740D35F0FA7B01021842
:101E0600273EF583ECF0A3EDF022900D4DEF75F033
:101E1600040217E2E412140890146FE025E024256A
:101E2600F822E0FF75F005A4F58285F0831213A76A
:101E3600540F22EF75F005A4FF9005F902180774F8
:101E4600FFF5F01214DDFCD3E5F09400EC64809409
:101E560080229013E4E0900D4D75F0041217E2E035
:101E660022EF900D4A75F0040217E23EF583E0FC7E
:101E7600A3E0FD2274802FF58274053E222DFFEE2D
:101E86003CFEF0A3EFF07C007D0502142AE0FE750F
:101E9600F02DA424E1F582E43401F583E5822F22B6
:101EA600FF9013AAE0FCA3E0FD22E0240CF582E4F7
:101EB6003413F583E022900001E92FF9EA35F0FAB0
:101EC60002151EEF25E02425F8760F0876FF2290EE
:101ED60013AAEEF0A3EFF022901481E025E0FF9024
:101EE6001480E033FE74B92FF582740422A804A985
:101EF60005AA06AB07E0FEA3E0FF22E025E024806A
:101F0600F582E43405F583E022FFE4FCFD02179434
:101F1600FF7B1FE4FCFDFAF9F80215DD7B017A0D63
:101F260079C29005F9021827E024DAF582E434052F
:101F3600F58322E47F2C7E01FDFC121753C30216A3
:101F4600FA9014A1E0FCA3E0FD22F583E4F0A3F0EF
:101F5600EF25E022E4F0EF24FAA3F0E0FD2461F897
:101F6600E6229005FAE475F0051214C790149EE077
:101F760004F02275F02DA424EFF582E43401F583F4
:101F8600E5822F22E9D36480F8740B64809822E0FE
:101F9600FEA3E0FFED25E02425F8A60608A6072205
:101FA60090147EEEF0A3EFF0229013E5EEF0A3EF8F
:101FB600F00D1214919013E5EE22900FB6E0D36463
:101FC6008022E4F0ED75F02DA42274172FF58274AB
:101FD6000622E4FCFD021794748F2FF58274062204
:101FE600EF25E02425F8E6FC08E622AB07AA06A9B9
:101FF60005A804021747E0A3FFE0FCA3E0FD22903A
:1020060013C5E0FF3395E0FEEF2274962FF5827438
:10201600003E22F0AF05125055EF4E22E4F0A374B5
:1020260005F022D39400EE9400221215D078051202
:102036001721AD07AC06229014711218078F82750E
:1020460083002274002FF58274002274532FF582C8
:10205600740622745A2FF58274002225E02425F88E
:1020660076080876002225E02425F8E4F608F6220C
:10207600E0FF740BD39F222470F58274053EF5832E
:10208600221217949013C60217479FEE6480F8EC4D
:0420960064809822A8
:10505500AD07EDB4010F121FC094807E0040037FA1
:1050650001227F0022EDB4020F121FC094817E0041
:1050750040037F01227F0022EDB4030F121FC0946D
:10508500827E0040037F01227F0022121FC0948090
:0B5095007E0040047F0180027F0022AB
:10575E00E4FFEF25E02400F582E43400121F50240C
:10576E00B9F582E43404F583E4F0A3F00FEFB42D21
:01577E00E149
:01577F002207
:1019DA00EF64116022EF6412601DEF641F6018EF5C
:1019EA0064206013EF6428600EEF642B6009EF64D3
:0C19FA00276004EFB42A03D38001C3224D
:1059500090130BE0FF7419D39F500BEF9426500661
:0C596000C3EF940EFF2290130BE0FF2217
:103EBA00E4FF121E107406F00FEFB405F5E4FF7468
:103ECA00612FF8E6FE900D51121E147402F0EE9066
:103EDA000D55121E6B7405F075F004EE900D591213
:103EEA0017E27405F074DA2F121F31E4F00FEFB401
:103EFA0004CDE4FF74FC2FF582E43405F583E4F085
:103F0A0074DE2FF582E43405F583E4F00FEFB41B79
:103F1A00E3E4FFEF25E02417F582E43406121F508C
:103F2A002453F582E43406F5837401F0A37490F007
:103F3A00EF25E0248FF582E43406121F50245AF547
:103F4A0082E43400F5837401F0A3742CF00FEFB40B
:023F5A001EC186
:013F5C002242
:1058F900121FE6D39400EC94004005EF12206C22AD
:0D590900900D4A121E13122022121EC922F8
:10571800121E67121E455011121E67121F52121FC9
:10572800E94C600EEF12206122121FE64C60031252
:035738001EC92265
:0247D500AE072D
:1047D700C2191219DA5032121DA3E06029121DA363
:1047E700121FC82406F582E43401121DAF121FC838
:1047F700240EF582E43401121DAF121FC82411F5EF
:1048070082E43401803702484E740BD39E501CEE6D
:1048170094185017121DA3E0600F121DA3121FC892
:104827002406F582E434018014801C121DA3E06085
:1048370016ED75F02DA424F8F582E43400121DAFAF
:0C484700E4F0AF050258F9AF0512571855
:014853002242
:0523600090146FEFF086
:10236500C20DC20EC20FE075F02DA424F8F9740059
:1023750035F0FA7B0190147112182790146FE090D4
:102385000D4C121DEBE0901470F0121E10E0B40617
:102395000D901470E0FF90146FE0FD0247D5901486
:1023A500701220765014EF9418500FEF64116004EA
:1023B500EFB41204D20F8002D20E300E4D12203D22
:1023C5001213A76015901470E0F582758300121E34
:1023D5001AE6FE08E64E7002D20D901470E0240E47
:1023E500FFE433FEA31218078F828E831213A770A2
:1023F500030224D58F828E83121E1AE6FE08E64E4E
:1024050060030224D5D20D0224D5200F030224B780
:10241500901470E064117048A3121807900011120F
:1024250013A7701890001F1213A7701090002712A1
:1024350013A7700890002A1213A76024900011E4D6
:1024450012140890001FE4121408900027E41214D7
:102455000890002A121E1AE6FE08E64E7002D20DFA
:10246500901470E064127068A3121807900012129D
:1024750013A770189000201213A77010900028124F
:1024850013A7700890002B1213A76044900012E464
:10249500121408900020E4121408900028E4121485
:1024A5000890002B121E1AE6FE08E64E7022D20D89
:1024B500801E901471121807901470E0FFF5827554
:1024C50083001213A7600912203DE4121408D20DEF
:1024D500300D0D90146F121DE7122022EF0225D743
:1024E50090146F121DE7121E4540030225D3121EDC
:1024F50067E4F0A3F0300E28901470E0FF121F027D
:10250500FCA3E0D39400EC9400505DEF25E0249CFF
:10251500F582E43405121DD7122029404D0225AF5E
:10252500200F030225BB901470E0FF6411703DD3AA
:102535009005A3E094009005A2E09400502A900530
:10254500D5E094009005D4E09400501C9005CFE0B0
:1025550094009005CEE09400500E9005BFE09400E5
:102565009005BEE09400400280408044EF64127004
:1025750064D39005A5E094009005A4E09400502A4A
:102585009005D7E094009005D6E09400501C900586
:10259500D1E094009005D0E09400500E9005C1E084
:1025A50094009005C0E09400400690146FE08016FA
:1025B50090146FE08014901470E0121DCE12202943
:1025C50090146FE040041220612212206C229014B6
:0525D5006FE0121ECAB8
:0125DA0022DE
:10189100C21AEF24FA90149FF0E0FF2461F8E69059
:1018A100149DF0125055EF4E60747B017A0D79C290
:1018B100121DDE121E45505F121E67E4F0A3F09068
:1018C100149EF090149EE0FFC39419503B121E3FEA
:1018D10012138E540F602C90149F121EB0FEF460F0
:1018E10022EF6E701E90149EA3121E93121DB4E07F
:1018F100600302196790149EE0121DCE1220294048
:1019010002D21A121F6880BB90149D121E21301A38
:10191100030219C30219C990149DE00219A290147F
:101921009FE075F07DA424C2F9740D35F0FA7B01B6
:10193100121DDE121E4540030219CE121E67E4F08D
:10194100A3F090149EF090149EE0FFC39419506987
:10195100121E3F12138E540F605990149F121E9342
:10196100121DB4E06012EE121E95121DB4E4F012C5
:101971001DE4122022EF802990149EE0FFEE121F39
:1019810079121DB4E0601EEFD3940A401890149EA2
:10199100A3E0121F79121DB4E4F0121DE4122022FB
:1019A100EF121ECA2290149EE0121DCE1220294071
:1019B10002D21A121F6802194790149D121E21307B
:1019C1001A06760808760022E4F608F62290149D9D
:0819D100121E21760F0876FFBB
:0119D90022EB
:09209A009013A4EFF0A3EDF0F99E
:1020A30012200925E0FBEE33FA745F2BF5827404EA
:1020B3003A121DD79013BA121F0F747B2BF582743B
:1020C300043A121DD79013BE121F0F121F8A40032A
:1020D30002235F9013A5E0FF6480949840030223DA
:1020E3005F1219DA500302235F9013A5E0F9FB3363
:1020F30095E0FAEB25E0FFEA33FE74052FF58274D1
:1021030004121E71745F2FF5827404121E0774216A
:102113002FF5827404121E71747B2FF582740412DE
:102123001E0774AB2FF5827403121E7174052FF50D
:10213300827404121E0774C72FF5827403121E7172
:1021430074212FF5827404121E0774512FF58274C3
:1021530003121E7174AB2FF5827403121E07746D84
:102163002FF5827403121E7174C72FF58274031244
:102173001E07121E7A121DD7FF9013AC121FD8EB45
:1021830025E0FBEA33FA749C2BF58274053A121DA1
:10219300D7FFE4FCFD9013B01217949013AC121701
:1021A3004774512BF58274033AF583EEF0A3EFF0F5
:1021B3009013B0121747AD07AC06121D95746D2F1F
:1021C300F5827403121E079013B01217479013ACD5
:1021D300121FF11215D09013B41217949013B41266
:1021E3001F39500302235F9013BE1217479013BA8F
:1021F300121FF11215D09013A61217949013A61262
:102203001F39500302235F9013BA121747780C1239
:1022130017349013A6121753125170121ED5901330
:10222300A5E0FF640B6004EFB4180C9013B87404BA
:10223300F0A374CBF0800A9013B87403F0A3743244
:10224300F09013B8E0FEA3E0121EA6D39FEC9E50BD
:1022530009E49013AAF0A3F080159013B8E0FEA34D
:10226300E0FFC3ED9FFFEC9E9013AAF0A3EFF09065
:1022730013A5E0FF640B6004EFB4180F9013ABE0F9
:1022830025E0F09013AAE033F080169013AAE0FE45
:10229300A3E0FF121E8C121ED57D0312143C121EE6
:1022A300D59013A5E0121D961220493E121DD71298
:1022B3001F169013AA121EF3E4FCFD122030901394
:1022C300A5E0121D96122049121E071220493E1244
:1022D3001DD7FF9013AAEEF0FCA3EFF0FD7B907ADD
:1022E300019013A4E0F9121D961220513E121DD73E
:1022F300C39DEE9C5011121EA7121D951220511260
:102303001D86121FD08027121D95121FD03E121D4D
:10231300D7121EA6C39FEC9E5017121D95121FD0F5
:10232300121E07ED2BFDEC3A121D94122051121EC2
:10233300079013A4E0FD121D96121FD03E121DD765
:10234300FF121ED5D394FFEE940F400A9013AA7484
:0C2353000FF0A374FFF09013AA121F9566
:01235F00225B
:053349009013C2EFF03B
:10334E00AF05EF121D97121E7AF583E0FFA3E090F2
:10335E0013CECFF0A3EFF0AF03EF121D97121E7A2C
:10336E00121DD7FF9013CFE02FFF9013CEE03EFE3D
:10337E00E4FCFD9013D0121794E47F1EFEFDFC902A
:10338E0013D0121F4050030234539013CEE0FEA30D
:10339E00E0FFE4FCFD780C121734A3121753125100
:1033AE00709013CA121FD89013CA121747780C12B6
:1033BE0017349013CA1217941220057802C333CE15
:1033CE0033CED8F912207D121747E47B3F121F1C13
:1033DE007806121721C004C005C006C0079013CA94
:1033EE001217477806121721D003D002D001D00051
:1033FE001215D09013C6122087C004C005C006C097
:10340E00071220057802C333CE33CED8F912207DB1
:10341E00D007D006D005D004122087E42FFFEE345B
:10342E0008FEE43DFDE43CFC780C121721D3EF942A
:10343E00FFEE940F40047E0F7FFF9013C2121E21E9
:05344E00A60608A60718
:013453002256
:105610007C007D0B12142AEEA2E713FEEF13FFC3EA
:1056200094CBEE648094845005E4FEFF80087435CA
:075630002FFF74FB3EFE2278
:0B52F100901480ECF0A3EDF0121FA65B
:1052FC00125610121FA6121EDE3E121DD7121F16BA
:10530C0090147E121EF3EE3395E0FDFC1220301249
:10531C001EDE121E07121EEB3E121DD7FF121FA619
:01532C00225E
:0D3CBE009014A0EFF0A3ECF0FEA3EDF0FFDA
:103CCB00AC02AD031252F19014A1EEF0FCA3EFF095
:103CDB00FD7B2C7A019014A0E0F9121D961220594D
:103CEB003E121DD7C39DEC6480F8EE648098501192
:103CFB00121F47121D95122059121D86121FDE80AE
:103D0B0028121D95121FDE3E121DD7FF121F47C32F
:103D1B001220905017121D95121FDE121E07ED2B4D
:103D2B00FDEC3A121D94122059121E079014A0E0BC
:103D3B00FD121D96121FDE3E121DD7FF9014A1EE31
:103D4B00F0A3EFF0D394FFEE6480948F400A9014AD
:0E3D5B00A1740FF0A374FFF09014A1121F9535
:013D69002237
:023D6A00A907A7
:103D6C00E4FBFAE9FD3395E0FCED25E0FFEC33FED6
:103D7C00122010F583E020E403023E08121F8A5043
:103D8C0025E964809498501EED25E0FFEC33FE7419
:103D9C009C2FF5827405121E71121E7A121DD72DDE
:103DAC00FFEE3CFE800A121D95121E7A121DD7FFE3
:103DBC00125610AA06AB07121D9574162FF58274B5
:103DCC00053E121DD7D39BEE9A50317C007D05AF7A
:103DDC0003AE0212142AAA06AB07EAC313FAEB13BA
:103DEC00FBD394FFEA940F40047A0F7BFFAD0312D0
:103DFC001D95122010F583EAF0A3EDF0AF01EF1240
:093E0C001D97122010121DD7FFB2
:013E1500228A
:1025DB00EF24FA9013E9121F60049013E4122019F0
:1025EB0070030226AA121F229013E9121EB0901339
:1025FB00E3F0F4700302268DE0FF641170030228F0
:10260B0049EF64127003022849121E3F75F005EF63
:10261B00121E2D7003022849900D65E0FF9013E701
:10262B00F0BF020B9013E4E0FF9013E30226F2904D
:10263B0013E7E0B404069013E30227009013E7E0DE
:10264B00640360030228499013E31220765013EFC2
:10265B009418500E121DBC9013E5121E83121FAF5F
:10266B00800D9013E3121F01FFA3E09013E5CFF051
:10267B00A3EFF09013E4121FFC9013E3E0FB7A003E
:10268B00801A900D65E0640360030228499013E4FF
:10269B00E0FF9013E3E0FB7A00E4FDFC023CBE900C
:1026AB0013E9121DF29013E9121F2EE09013E8F0BC
:1026BB001259509013E3EFF064117003022849E0B4
:1026CB00FF64127003022849121E3F75F005EF12CA
:1026DB001E2D70030228499013E4E0FF121E5C903C
:1026EB0013E7F0B40206A3E0FD02209A121E58B4C1
:1026FB0004149013E8E0FF123D6A9013E4121E21BC
:10270B00A60608A60722121E586403600302284976
:10271B009013EBF0A3F0A3F0A3F09013E9E0900576
:10272B0013121DF6E49013EAF09013EAE0FFC36472
:10273B0080949940030227F3900513121807EF3387
:10274B0095E08F82F58374051217D11213A7540FDE
:05275B0070030227EAF3
:102760009013EAE0FD121D96121E7AF583E0FFA396
:10277000E09013EFCFF0A3EFF0ED121F8B503290EB
:1027800013EAE0FF648094985027EF121D97749C21
:102790002FF58274053E121DD7FF9013F0E02FFF36
:1027A0009013EFE03EFE9013E5121E88121FAF80DB
:1027B0000B9013EFE0FFA3E09013E5CFF0A3EFF051
:1027C0009013EBE0FEA3E09013E5121FFED312205E
:1027D0009040179013EBECF0A3EDF09013EAE0FEBD
:0A27E0003395E09013EDF0A3CEF066
:1027EA009013EAE004F00227349013E4E0FF901318
:1027FA00EBE0FCA3E0FDA3E0FAA3E0FB123CBE3051
:10280A00093DE49013EAF09013EAE0FFC364809470
:10281A00AD502AEF3395E0FE74112FF58274133E02
:10282A00F583E070109013EAE0121D97121E7AF5F4
:0F283A0083E4F0A3F09013EAE004F080CAC2092F
:01284900226C
:10442700901484121F5A2402901483122019602FAB
:10443700121F22901485121EB0FFF4606790148239
:10444700EFF0121E3F901482121E286057121E3979
:10445700121EBC1244ACC333CE33CED8F980399088
:104467001485121DF2901485121F2EE0901484F00B
:10447700125950901482EFF0121E3F901482E012EE
:104487001E2A6020901484E0121E3A121EBC1244A9
:10449700ACC333CE33CED8F9FF901483121E21A6B6
:0444A7000608A60756
:0B44AB0022FFAEF01250E8EF78022272
:103A8600901488121F5A2403901487122019604D2F
:103A9600121F22901489121EB0FFF47003023B48D5
:103AA600901486EFF0900D6DE064057025121E3FB0
:103AB600901486121E287003023B48121E3990008D
:103AC60003121EBFAEF07802C333CE33CED8F9024E
:103AD6003B30901487E0FF901486023B4390148994
:103AE600121DF2901489121F2EE0901488F01259BC
:103AF60050901486EFF0121E3F901486E0121E2A94
:103B06006040901487121E5BB4052C901488E01256
:103B16001E3AE92FF9EA35F0FA90000312151EAEA7
:103B2600F07802C333CE33CED8F9FF901487121E35
:103B360021A60608A60722901487E0FFA3E0FD123F
:023B4600209AC3
:013B4800225A
:0541D200901474EFF0F1
:1041D700900D4C121E5F901478F01259509014777E
:1041E700EFF0901474E0FF121E5CB402089014788C
:1041F700E0FD02209A901474121E5BB4041B901405
:1042070078E0FF901477E06F7058123D6A9014744D
:10421700121E21A60608A6072290147812207650AF
:1042270020EF9418501B121DBC901475121E83901A
:104237001475EEF0A3EFF00D12143C901475EE8098
:104247000D901478121F01FFA3E0901475CFF0A30F
:10425700EFF0901474121FFC901478E0FB7A0012B0
:024267003CBE5B
:014269002232
:1050E8007B69121F1990148A12179490148A121748
:1050F80047E47B64FAF9F812166890148A12179438
:10510800E47FFF7E0FFDFC90148A121753C3121719
:1051180010400A90148A1217A000000FFF90148AFA
:0351280012174714
:01512B002261
:105A8500781DE0FEA3E0A60608F62292AFAF028FCE
:065A9500B1AF038F842273
:104C0C00AB84AAB1A2AF921B90148E12179490147D
:104C1C0090125A8553B10F90148FE0700543B11068
:104C2C008019901490E030E70543B130800D43B10A
:104C3C0020901490E04480F0125A85E4F584C2AFC1
:104C4C0043B701758F03781DE6FE08E6F5828E8367
:0C4C5C00E4F053B7FEF58FA21B125A9033
:014C68002229
:1048D000AB84AAB1A2AF921C901416121794901434
:1048E00015E0F9FF3395E0FEEFF44E605390141895
:1048F000787D125A8753B10F901417E0700543B1B9
:10490000108020901418E030E70543B13080144344
:10491000B120901418E04480F0E0FEA3E0787DA67A
:104920000608F6E4F584C2AF43B701758F01787DC0
:10493000E6FE08E6F5828E83E9F053B7FEE4F58FD4
:05494000A21C125A90B8
:01494500224F
:105B9C000001FF00FF000001010000FF00FF0100F9
:1053DA00E56785688385698222901493021807D34A
:1053EA00ED9408EC6480948022D3ED9410EC6480F0
:1053FA00948022C3ED94F8EC6480947F22C3ED94E8
:07540A00F0EC6480947F22A6
:054A8200901492EFF01A
:104A8700E5662401FFE43565FAA9077B01A312183F
:104A9700271253E374019013056B7008E965827060
:104AA70003EA6583700C7B017A127985901493125F
:104AB70018271253E31253DA6B7008E96582700303
:104AC700EA65836019901492E0856682856583F0B4
:0E4AD7001253E3AF018A658F66901492E0F0EF
:014AE50022AE
:104ED40053E6F7AA65A9667B011253DA6401700AE6
:104EE400E56665827004E56565837003FF802B7851
:104EF40067E475F0011217F712138EFF7401901313
:104F0400056567700AE56965827004E56865837004
:0D4F14000975670175681275698543E60827
:014F2100226D
:1056370053E6F71253DA6401700AE566658270046F
:10564700E56565837003FF800AAB67AA68A96912DD
:06565700138EFF43E6087C
:01565D00222A
:031A1E00022AAAEF
:102AAA00C0E0C0F0C083C082C0D075D000C000C0F2
:102ABA0001C002C003C004C005C006C00790126866
:102ACA00E06003022CA130DF02C2DFE5B05407F553
:102ADA006C656A600CE56C656AF56E756B03856CEE
:102AEA006AE56B603A156BE56B7034E56E30E00AA7
:102AFA00E56C20E0057F01124A82E56E30E10AE5C5
:102B0A006C20E1057F02124A82E56E30E211E56C23
:102B1A0020E20C9012807401F0A374F4F0D2103009
:102B2A00102E90128074FFF5F01214C7901280E0F4
:102B3A007002A3E0700EC21090133EE0FF7D1312E4
:102B4A0057E3800CE5B030E207C2107F04124A82D4
:062B5A0020D90330D85C15
:102B6000E5901313543F9014B4F0C2D8C2D9901218
:102B700084E0FF9014B4E0FD6F5403603FEF75F004
:102B800004A47E00540CFFED5403FDEF4D249CF58E
:102B900082EE345BF583E4939014B5F06016E0FFA9
:102BA0003395E09012828FF01214C790127EE4F0F9
:0C2BB000A37405F09014B4E0901284F0BF
:102BBC0090127EE07002A3E0600A90127E74FFF522
:102BCC00F01214C790127EE07004A3E0640160035D
:102BDC00022CA1901282E0FCA3E0FD64024C700573
:102BEC007F05022C971253E950047F0180027F006D
:102BFC00901282E0FCA3E0FDD39402EC64809480FC
:102C0C0040047E0180027E00EE5F60057F07022C8F
:102C1C00971253F350047F0180027F001253E94056
:102C2C00047E0180027E00EE5F60047F09805C12EE
:102C3C0053F340047F0B8053BCFF07BDFE047F069B
:102C4C0080491253FD40047F0180027F00C3ED9444
:102C5C00FEEC6480947F50047E0180027E00EE5F67
:102C6C0060047F08802512540740047F0180027F96
:102C7C00001253FD50047E0180027E00EE5F600462
:102C8C007F0A8007125407500C7F0C124A82901254
:102C9C0082E4F0A3F0D007D006D005D004D003D046
:102CAC0002D001D000D0D0D082D083D0F0D0E0328E
:1059F4007B017A1279858B678A6889698A658966E9
:0A5A0400E4901280F0A3F0C210221B
:105B4200E475F0011214DD85F082F58322EEF0A3F4
:045B5200EFF0A322AB
:0B5C1A00AF01AE027C00E4FD024C0C68
:055AC6009014C9EDF091
:105ACB00AF01AE027C00E4FDE0901415F00248D06B
:104E2900901457125B4FECF0A3EDF0A3EAF0A3EB5B
:104E3900F090145BE07002A3E0603A901457E0FE32
:104E4900A3E0AA06F97B01A3E0FEA3E0F5828E8325
:104E5900E0FD125AC690145B74FFF5F01214C79066
:104E69001459E475F0011214C7901457E475F00150
:064E79001214C780BC22E8
:085C5800E49006CBF0A3F0225A
:10556A009006CBE0FEA3E0AA06F97BFF125C1A9034
:10557A0006CBE0FEA3E0FF7C067DCD7B007A041219
:0A558A004E29E49006CBF0A3F022B6
:0D46520090143DEDF090143BEEF0A3EFF05E
:10465F00EE54FCFE9006CBE0FCA3E0FD7002EE6C86
:10466F006044ED4C600312556A90143BE0FEEE542B
:10467F00FCFE7F009006CBF0A3EFF090143E125B90
:10468F004F7406F0A374CDF07FFF7E0390143E129B
:10469F005B42E493FD901440125B42EDF0EF1F700C
:1046AF00011EEF4E70E690143DE0FF90143BE0FCCE
:1046BF00A3E0FDEC5403FC74CD2DF58274063CF59C
:0346CF0083EFF086
:0146D20022C5
:1053A200901442125B4F12182790144774FFF5F0C5
:1053B2001214DD45F06020901442E475F0011214DD
:1053C200DDAFF0FE901444E475F0011218101213D0
:0853D2008EFD12465280D2222A
:104F22000001020408100000030418000000000041
:104F32001F00000000001804030000000010080415
:104F420002010000040A0A11110000010102021C00
:104F520000001C02020101000010100808070000F6
:0E4F62000708081010000020406080A0C0FF6B
:0D5BD9007F147E00EF1F70011EEF4E70F76D
:015BE600229C
:105B8B007F381258437F061258437D0EE4FF025CA8
:015B9B000207
:055843009014CAEFF013
:10584800A2AF921DC2AF1257C3EF20E7F99014CA56
:09585800E0FF125881A21D92AF7D
:015861002224
:1057C300A2AF921EC2AF75A0FFC2B5D2B6D2B712B6
:0F57D3005BD9ADA0C2B7125BD9A21E92AFAF05D2
:0157E20022A4
:055CB3007F01025843CF
:10588100A2AF921FC2AF8FA0125BD9C2B5C2B6D26E
:0D589100B7125BD9C2B7125BD9A21F92AF4C
:01589E0022E7
:1059A400A2AF9220C2AF8FA0C2B6D2B7D2B5125B5B
:0A59B400D9C2B7125BD9A22092AF4E
:0159BE0022C6
:0C5C02009014CBE05FF04DFFF00258431F
:025A0E00AC07E3
:105A1000A2AF9221C2AF1257C3EF20E7F9AF041231
:065A200059A4A22192AF7F
:015A2600225D
:1056AC009014A31218279014A312180712138E60CB
:1056BC00139014A3E475F00112181012138EFF123C
:0556CC005A0E80E222ED
:0653680090145D121827ED
:10536E00A2AF9222C2AF125CB3E4FDFF125C0E90AC
:10537E00145D1218071256ACE4FD7F01125C0E90FC
:10538E0014601218071256AC7D107F01125C0EA22B
:03539E002292AFA9
:0153A10022E9
:0C5C0E00EF75F040A42D2480FF025843E5
:0B5C2500E4F584EF904F6893F5D32264
:0B409D0090140AEDF090140712182791
:1040A800AF0190140FEAF0A3EFF090140B74FF1215
:1040B8001761EC4D4E4F6078901407121807E924E9
:1040C80028F9E43AFAC003C002C00190140FE0FED8
:1040D800A3E0FFF9D082D083D0E064017008E965DD
:1040E800827003EE65836020901407121807E92494
:1040F80042F9E43AFAEB8A83898264017008EF6531
:10410800827003EE658370098F828E837404F08059
:104118001290140AE0FF90140FE0FCA3E0F5828CE3
:1041280083EFF090140FE475F0011214C70240B247
:014138002264
:1057E3009014B6EFF0A3EDF07F0A124C699014B653
:1057F300E0FF124C699014B7E0FF124C69025BE7BB
:085C60007F02124C69025BE7B0
:0654B500121A09EF602746
:1054BB009014B87414F0A37449F01255BE9014B83C
:1054CB00E475F0011214DD85F082F583EFF0121A0A
:0754DB0012EF70E67F0122D1
:0354E2007F002226
:105ADB009014CCEFF07F2F124C699014CCE0FF1296
:055AEB004C69025BE7BD
:105AF0009014CDEFF07F30124C699014CDE0FF127E
:055B00004C69025BE7A7
:1036590090650175F070ED1217E2EC75F070A42514
:1036690083F8ED25E028AF829013E0F0A3EFF09006
:1036790013D8E0FF7E007C027D7012142A74012F9A
:10368900F974653EFA7BFF22E0FF75F070906501E1
:103699001217E2EF25E02583AF8222900D45E475EC
:1036A900F0010214C7FE7A0D794A74027B01901465
:1036B90047F0A322900ACEE475F001121810AE0269
:1036C900AF0122E024FFFFE434FFFE9013D9E0FCB0
:1036D900A3E0FD22900D45E0FCA3E0FDC39470EC4E
:1036E900940222E475F0011214DD85F082F583E479
:1036F900932224FFFEE434FF9013D9F0A3CEF022E5
:103709009013DD121827E49013DBF0A3F022AD0427
:10371900EDFFEEF0A3EFF022E4900D45F0A3F022C7
:10372900AF05E4F0A3EFF0E07F00FE2274D32DF59E
:1037390082740A3CF583229FEE6480F8EC648098D9
:01374900225D
:104E7F009014BA7402F0E4A3F0125C587E657F00C0
:104E8F007A1479BAE41236B504F01253A27EB07FC9
:104E9F00917B017A1479BB901447E4F0A304F012CC
:104EAF0053A212556A7B017A0D794A90140B12178F
:104EBF00A000000270E4FD12409D123EBA125A404B
:054ECF007F1E02532DBF
:105A270090B091E493600C906500E4936402600386
:095A3700124E7FE4900D48F022AC
:05532D009014BCEFF03C
:10533200125C58E49014BDF09014BCE0FFA3E0FEB0
:10534200C39F501F75F070EE9065011217E2EE12C6
:10535200369D1236AE7470F01253A29014BDE00462
:06536200F080D502556A3F
:0F5BCA00300B06125C60D21222D20A12355B2217
:031A1B00025BCAA1
:1054110090142312182790142974FFF5F01214DD4B
:1054210045F0602290142612180712138EFF901473
:1054310023121807EF1213F69014241236A79014B2
:07544100271236A780D022DC
:10559400900D4CE09014CEF0900D4812367B901490
:1055A400261218279014297402F0A37470F07B015A
:0955B4007A0D794A125411C21259
:0155BD0022CB
:105B0500125C58900D481236911236AE7470F01230
:055B150053A202556AD5
:105A4000A2AFE4339014CFF0C2AF125B05C2129044
:075A500014CFE024FF92AF28
:015A5700222C
:08382A009013D4EFF0A3EDF0C0
:10383200A2AFE4339013E2F0C2AF9013D4E0FFD30F
:103842009B4033EF1236FBEB149013D8F09013D554
:103852001236CCD312374050581236591237091249
:1038620038BC40FB12556A9013D91236A79013D870
:10387200E004F002384F9013D5E01236FB9013D7D4
:10388200E014A3F09013D41236CCC3123740402177
:103892001236591237091238BC40FB12556A90137E
:1038A200D974FFF5F01214C79013D8E014F002385F
:0938B200869013E2E024FF92AFBE
:1038BB00229013DDE475F001121810AE02AF0190E7
:1038CB0013E0E475F0011214DD85F082F583E493C7
:1038DB00FD1246529013DBE475F0011214C7C3902E
:0C38EB0013DCE094709013DBE0940222E8
:0538F700900ACDEDF088
:1038FC00A2AFE433900D47F0C2AFEF14900D43F03C
:10390C00EB14A3F0900ACDE014FF900D43E0D39F8D
:10391C0040030239B6A3123691FE1237211236DD5E
:10392C0050190FEFAA0670010E14F5828A83E493E6
:10393C00FB123735EBF01236A480E2900D441236B0
:10394C007B900ACE121827900D43123691900AD113
:10395C00F0A3EFF01237211236BD900AD11236ECDB
:10396C00FD1246521236A4C3900D46E09470900D91
:10397C0045E0940240E1900D4312367B900ACE1242
:10398C0018271237211236DD50101236BD1237357A
:10399C00E0FD1246521236A480EB12556A900D438C
:1039AC00E004F0A3E004F0023910900D47E024FF8E
:0239BC0092AFC8
:0139BE0022E6
:07426A009013FCEBF0AC0720
:10427100A31237299013FDF0A3EFF09013FD12372D
:1042810017A2AFE433901406F0C2AF901405740F77
:10429100F0125C5890140512367B90140112182705
:1042A100E49013FFF0A3F09013FDE0FCA3E0FFEC1A
:1042B100FD9013FCE0FBE4901499F0D21412374AFC
:1042C100901404EFF0FD9014011236C01246529082
:1042D10013FD1236A79013FF1236A7C3901400E006
:1042E10094709013FFE0940240BD12556A9014053A
:1042F100E004F0E0C3941E4098125277D2AF025C02
:014301004F6C
:0741390090141AEBF0AC0733
:10414000A2AFE433901422F090141D12372990147A
:104150001DF0A3EFF090141D123717C2AF90142179
:10416000740FF0901421E0FFC3941E505675F07048
:10417000EF12369690141FF0A3EFF0E490141BF0AA
:10418000A3F090141DE0FCA3E0FFECFD90141AE0F6
:10419000FB90141F1236EC901499F0C21412374A97
:1041A00090141D1236A790141B1236A7C390141C2E
:1041B000E0947090141BE0940240C7901421E00436
:1041C000F080A0125C4F125277901422E024FF92EC
:0141D000AF3F
:0141D10022CB
:07374A00901496EFF0A905B1
:10375100C21520C3FD20C5FAC2C4D2C5E4FFFD30A5
:10376100C3FD30C3FDE5C154F8FC64086004ECB44A
:103771001013EFB40105EB44018003EB54FEF5C2D5
:103781007D01023818ECB4180B89C27D02C2C4C293
:10379100C5023818ECB420028045EC6428703CED79
:1037A100B4020E901496E0F5C27D03C2C5C2C48076
:1037B10066EDB4031B301408D2C57F01C2C4805723
:1037C100901499E0F5C2C2C57D04E4FFC2C48047EC
:1037D100ED64047042D2C47D05803CECB4300AD261
:1037E100C4D2C57D08E4FF802EECB438028024ECFD
:1037F100B44006C2C2C2C5801EECB448028014ECBB
:10380100B450028004ECB4580AD2C47D07AEC2C2DF
:10381100C28004D2C4D2C5C2C3ED64076008ED649E
:08382100056003023763AF06E6
:01382900227C
:10589F007E0F7FDD8E738F748E6F8F707E107FA55E
:0E58AF008E758F768E718F72E4F577C223228C
:031A0F0002494643
:10494600C0E0C083C082C0D0309821C298857082F2
:10495600856F83E599F00570E5707002056FB4A563
:104966000BE56FB41006756F0F7570DD309937E57E
:0349760077602F38
:10497900857682857583E09014D0F0C299F5999077
:104989000FBAE599F015770576E57670020575B4E5
:0D4999006D11E575B4110C7575107576A5DE
:0F49A6008004C299C223D0D0D082D083D0E03217
:105B6800E57065747004E56F657360037F01227FDB
:025B7800002209
:10586200857482857383E0FF0574E57470020573A5
:0E587200B4A50B7410B5730675730F7574DD55
:015880002205
:0A4A420041134E0041136700C11735
:1051B400901351E475F0011214DD85F082F5832219
:1051C4009013517413F0A37468F022901348E4759B
:1051D400F0011214C77E137F7C901348E0229013D1
:1051E4004CE0FFA3E090134822E0F5C2901348E09E
:0251F4006E2229
:10596C00AF84E4F584C2C343E60243F60275C30177
:0B597C0075C04475CF8F43C3018F84BA
:0159870022FD
:105277007E137F5390134AEEF0A3EFF090134FEE97
:10528700F0A3EFF0901346EEF0A3EFF07E137F68E4
:1052970090134CEEF0A3EFF0901351EEF0A3EFF064
:0D52A700901348EEF0A3EFF0C21602596C10
:10565E0090134F1251B7EFF090134F1251B7EDF068
:10566E0090134FE0B4130FA3E0B4670A90134F7476
:07567E0013F0A37453F022A6
:0D5BE700AF84E4F584C216C2C4D2C58F8419
:015BF400228E
:104C690020162FD2161251B474FFF07C137D7C905C
:104C79001351E0B50408A3E0B505031251C412515C
:104C8900B4E4F0901351E0B50408A3E0B5050312AC
:104C990051C41251B4E4F0901351E0B41308A3E0E5
:104CA900B47C031251C41251B4EFF0901351E0B423
:0D4CB9001308A3E0B47C031251C47F012254
:1055130090134AE0FCA3E0FD901346E0B50408A312
:10552300E0B505037F002290134AE0FCA3E0F58277
:0C5533008C83E0B507037F01227F00227B
:1055BE0090134AE475F0011214C790134A1251B7B2
:1055CE00E0FF90134AE0B4130FA3E0B4670A901300
:0855DE004A7413F0A37453F0AA
:0155E60022A2
:061A09007FFF12551322BD
:061A1200E4FF125513224F
:031A180002307821
:10307800C0E0C0F0C083C082C0D075D000C000C01E
:1030880004C005C006C007E5C154F812185C31E059
:103098000030D30830D31030FC18312320312928D0
:1030A800318B30319038319A50319A5831A660318D
:1030B8009C6831A670319C78319A8031B588319AF4
:1030C8009031B59831C8A00000320DC2C51251CF59
:1030D800B5060BA3E0B507069013481251C7901325
:1030E800481251B71251ED7003A3E06F600302322A
:1030F8000D0231821251CFB5060BA3E0B507069039
:1031080013481251C79013481251B71251ED70036A
:10311800A3E06F600302320D0231821251E2CF80C8
:103128001B901351E0FEA3E0FF901348E0FCA3E0DE
:10313800FDB50713ECB5060F90134CEEF0A3EFF0B6
:10314800C2C5D2C402320D8D828C83E0B4FF07C29F
:10315800C4D2C502320D1251CFB5060BA3E0B50794
:10316800069013481251C79013481251B71251EDE7
:103178007003A3E06F600302320D9013481251C729
:1031880002320D1251E2802F1251E2CFF0A3EFF07C
:10319800807380101251E2CFF0A3EFF0D217ADC2C6
:1031A8007FFF8004ADC2E4FF12565E80589013463C
:1031B800E0FFA3E090134FCFF0A3EFF0D2C4804517
:1031C80090134FE0FFA3E0901346CFF0A3EFF03049
:1031D8001733D2C5C217802D90134CE0FEA3E0FF31
:1031E800901348EEF0A3EFF0901346E0FDA3E090B3
:1031F800134FCDF0A3EDF0D2C4A3E06E7003A3E0AB
:103208006F6002D2C5C2C3D007D006D005D004D0A3
:0C32180000D0D0D082D083D0F0D0E032C3
:102CBC004C00500049002000540043560050756CE5
:102CCC007320313A2573257320323A25732573000E
:102CDC00333A2573257320343A2573257320353AFE
:102CEC00257325730043562031303A257325732004
:102CFC0031313A257325730031323A25732573200F
:102D0C0031333A2573257331343A257325730043D7
:102D1C006F6E747261737420256420006F66660098
:102D2C00363700363738003637383900506F6C7903
:102D3C0070686F6E792025732000546F67676C651F
:102D4C00005375737461696E004C3A2573202563CA
:102D5C00657600523A257300526164696F3A2564B6
:102D6C002025733A257320257320004B59006B796D
:102D7C00004356313A252D3364204356323A2564AC
:102D8C0020004356313A252D3364204356323A25E0
:102D9C007320006C6F6300616263646566676869C9
:102DAC006A6B6C6D6E6F70717273747576777879FF
:102DBC004142434445464748494A4B4C4D4E4F507F
:102DCC00515253545556575859FF2CBC02FF2CBE28
:102DDC0003FF2CC004FF2CC200FF2CC406FF2CC622
:102DEC0005FF2CBC020006000700080009000500C6
:102DFC0009000D00110007FF5CB80008FF5CAD0076
:102E0C000CFF5CBD000DFF5C8B0102FF5CC201037B
:102E1C00FF5C920107FF5CC70108FF5C99010CFF86
:102E2C005CCC010DFF5CA00006FF32240008FF59AA
:102E3C0088000BFF5448000DFF44B60105FF5009F4
:102E4C00010DFF47540006FF5CD10007FF5C6800D2
:102E5C000CFF5CD6000DFF5C6F0103FF5CDB010413
:102E6C00FF5C760109FF5CE0010AFF5C7D010EFF4F
:102E7C005CE5010FFF5C840009FF5A9B0109FF5AB6
:102E8C009B000AFF5780010AFF57800002FF5C304D
:0A2E9C00000AFF573B0102FF5BF53F
:104A4C004311AE00000041126202C1254112670100
:104A5C0041123900411268000C0FFF2D28FF2D2C3C
:104A6C00FF2D2FFF2D330609FF2D46FF2D4D01087D
:054A7C0001021B000116
:10284A00EDFF3395E0FE75F003EF1217E2EE75F037
:10285A0003A42583F5832224A3F9E4342DFA12185C
:10286A002702138E7A12794F9014607B011218276F
:10287A007A12793C2290117D75F003ED1217E2EC81
:10288A0022EFF0A2AFE433A3F012553FC2AF901289
:10289A00687401F0EF75F005A4FF9011AE021807F5
:1028AA007BFF90137F0218279011AE1218279012FF
:1028BA0039E075F002A4FFAEF024F1F9742D3EFA66
:1028CA007BFF9011B602182712180712183C9013B2
:1028DA00821218277B0122E024A3F9E4342DFA227C
:1028EA00FD9012691218071214F3AEF078022290C2
:1028FA0011B112180702138E12180712183C9013FE
:10290A008802182790142C12180774021213F67BE7
:10291A00FF7A2D79D5227BFF90119D0218277B0122
:10292A009011B10218277B017402AD0790147DF053
:10293A002290143512180790000322121807902DBE
:10294A00BBD3E99582EA95832274031213F67BFFBF
:10295A007A2D79D922F9E4342DFA7BFF90127B0281
:10296A001827901382F0A3EFF022EDFF3395E0FED3
:10297A002275F005EFA429F9EA35F0FA02138E90D0
:10298A0011CD021827EFF09011B61218070214F3AE
:10299A002479F9740D3EFA7B01021827D3EF64807B
:1029AA00948022901453E0FFA3E0901382CFF0A307
:1029BA00EFF02212180712183C90138E1218277B78
:1029CA00012275F003A4246FF582E43412F5832200
:1029DA0075F005A424D2F582E43411F5832275F04A
:1029EA0005A424D0F582E43411F5832275F005A4F8
:1029FA0024D1F582E43411F58322E075F07DA42414
:102A0A00C2F9740D35F0FA22E0FEA3E090117D754B
:102A1A00F00322901267F07BFF227BFF7A2D79DD8B
:102A2A002212151EFFAEF0D39400EE94FE229013EC
:102A3A008502182774F92FF9742D3EFA901269222B
:102A4A00121807C3E994A322900FB6E0C364802248
:102A5A00E075F003A42409F80217EEE024FF92AF10
:102A6A00E4901268F0229013911218277A12794F83
:102A7A0022244DF582740D3EF5832212180774FF45
:102A8A00902DB46B2212180774FF902DB56B222477
:102A9A0051F582740D3EF583227B017A12793C222C
:10454500E490119CF090119BF09011A2F09011A1B4
:10455500F09011A0F09011A3F07B017A0D79C29033
:1045650011AE1218277BFF7A2D79F11228CC7A2DFE
:1045750079F99012691218277A2D79A390127B1276
:1045850028689011B9F0E4A3F0901234F0FF1229D5
:1045950019EF1229CC1218270FEFB404F1E4901289
:1045A5003BF090124EF0901261F0901264F0901270
:1045B50066F09011A5F09011A7F09011A9F0901157
:0645C500ABF09011ADF017
:0145CB0022CD
:065CA700E49011B5F022AB
:104B49009014BEEEF0A3EFF0AF051DEF6053901483
:104B5900BEE0FEA3E0F5828E83A3A3121830901164
:104B6900B5E0FF1229DA1218279014BEE0FAA3E083
:104B7900FBF5828A83E493FEEF1229E8EEF08B823B
:104B89008A83740193FF9011B5E01229F6EFF09032
:104B990011B5E004F09014BEE475F0051214C78055
:024BA900A72241
:1057A2001228F9FE1229E8E0FFEE1229F6E0FD12B6
:1057B2005C0E1228F91229DA1218079011CA02187F
:0157C20027BF
:1059BF009011B112180774011213D41228F9FF9025
:0B59CF0011B5E0B50704E41213F62246
:1055E700D3ED6480948040047401800274FF121329
:1055F700D412138EFFB4FF03E4800A90147DE0FEFB
:09560700B50705EE141213F6229A
:105A9B007B017A12796274081229341255E790123D
:065AAB0062E0FF025C2531
:105780007B017A0F79B6AD0790147D7404F0125541
:10579000E7E4901239F0122A041228B2122A3E02CB
:0257A0001827C8
:0B5C30007A0F79B71229301255E722D5
:10573B007A0F79B91229301255E7E4901306F090DD
:10574B001343F07F05125A587F011259DA7F031267
:03575B0059DA22F6
:0D5BF5007B017A0F79B81229321255E72290
:095C4F0090119D12180702188241
:1058BD009012677401F07A4879541229207A587938
:0E58CD00DB1229897A5979BF90126C021827D4
:1058DB009012677402F07A2E79A61229207A5979E0
:0E58EB00161229897A5979BF90126C0218277B
:105916007403122A1D7A4379961229227A59793309
:0D5926001229897A5979BF90126C02182756
:105933007404122A1D7A5079A01229227A58790305
:0D5943001229897A5979BF90126C02182739
:105803009012677405F07BFF7A5279381229227A55
:105813005879231229897A5979BF90126C02182773
:105823009012677406F07BFF7A4A79E61229227A8E
:105833005879BD1229897A5979BF90126C021827B9
:0251F600AD0703
:1051F800ED3395E0FEEF7802C333CE33CED8F99085
:10520800146312299AAF05EF3395E0FE90115012FE
:105218002850121807901466121827901463122841
:10522800FCB40209122953901466121827021A1B9B
:1052B4001229A67BFF40067A2D79E580047A2D79A0
:1052C400E19011BB12284A1218271229749011BBBD
:1052D40012285012293E1213A7FCEF7802C333CED2
:0D52E40033CED8F9122A7BECF0121A1B22EF
:055CB800E4FD0252B4FE
:055CBD007D010252B45C
:055CC2007D020252B456
:055CC7007D030252B450
:055CCC007D040252B44A
:1046D30090142C1218271229A6402690142C122865
:1046E300FC24FE600A1460091460062404705F80D1
:1046F3002490142C12180774041213F6122A24801F
:104703004790142C1228FC24FE600F1460111460CF
:104713002E24047039122953802E12290E802990D9
:104723001432E075F003A4246EF582E43411F583AA
:104733001228FCD3648094EB401412290E80099054
:10474300142C12180712295390142F121827021A27
:014753001B4A
:02512C00AC07CE
:10512E00122974EF7802C333CE33CED8F9901469B6
:10513E0012299A12297490115012285012180790A1
:10514E00146C121827AF0490146C12180790142FB9
:10515E00121827901432EDF09014691218071246A7
:01516E00D36D
:01516F00221D
:055CD1007D0A02512CC8
:055CD6007D0B02512CC2
:055CDB007D0C02512CBC
:055CE0007D0D02512CB6
:055CE5007D0E02512CB0
:1039BF001229A6404312287F122858A3E475F0015C
:1039CF001214C730247C12287F122858122A8570AF
:1039DF0008E965827003EA6583601512287F122853
:1039EF0058122A8F7008E965827003EA6583705256
:1039FF007BFF7A2D79B6804112287F122858A37445
:103A0F00FFF5F01214C730243912287F12285812EC
:103A1F002A857008E965827003EA658360151228AC
:103A2F007F122858122A8F7008E965827003EA65A1
:103A3F0083700F7BFF7A2D79B312287F12285812CB
:103A4F00182712287F12285812294540087BFF7A21
:103A5F002D79BB801812287F122858121807C3908F
:103A6F002DA312294C500F7BFF7A2D79A312287F9B
:073A7F00122858121827223B
:104D21009014C0ECF0A3EDF0D2241239BF9014C05E
:104D3100122A12122854122A4AFD9014C0E0FAA332
:104D4100E0FB7802C333CE33CED8F9248CF58274DC
:104D51000D3EF583EDF0122A16EB1217E2EA122846
:104D6100581228FCC3648094EC500B9014C0A3E04B
:094D71002405FF1251F6021A1B81
:075C68007D057C00024D21C7
:075C6F007D067C00024D21BF
:075C76007D077C00024D21B7
:075C7D007D087C00024D21AF
:075C84007D097C00024D21A7
:10547F009014C2ECF0A3EDF0C2241239BF9014C205
:10548F00122A12122854122A4AFD9014C2A3E0784D
:10549F0002C333CE33CED8F9244CF582740D3EF5CA
:0654AF0083EDF0021A1B60
:065CAD00E4FDFC02547F3F
:075C8B007D017C0002547F43
:075C92007D027C0002547F3B
:075C99007D037C0002547F33
:075CA0007D047C0002547F2B
:103224001229A650030232AA1228A47401900DC2D6
:103234006B7008E965827003EA6583701F900FB6AE
:10324400E014601014601014600F24036003023350
:103254003702330302332A806902330B1228A47421
:1032640001900E3F6B7008E965827003EA65837014
:103274000302332A1228A47401900EBC6B7008E96F
:1032840065827003EA6583700280371228A4740192
:10329400900F396B7008E965827003EA65836003F7
:1032A4000233370233331228A47401900DC26B70B9
:1032B40008E965827003EA65837011122A529483C7
:1032C40050089012397403F08069803B1228A4746A
:1032D40001900E3F6B7008E965827003EA658370A4
:1032E40002804C1228A47401900EBC6B7008E9652E
:1032F400827003EA65837012122A529481500890F6
:1033040012397401F0802CE480251228A4740190F1
:103314000F396B7008E965827003EA6583701412D3
:103324002A52948250089012397402F08005E49075
:103334001239F0901239122A047B011228B2122A8F
:053344003E12182722D3
:105988001229A640079012387401F022E4901238C8
:0C599800F07F03124CC67F39125A5822CF
:10553F0090127B121807C3902DA312294C40109084
:10554F00127B122945500890127B122A4AFF229093
:0B555F00127B121807C3E994BCFF2266
:02544800AE07AD
:10544A0012553FD3EE64809480401274BC2F122907
:10545A005F1228A412297B54F04401801274A32FEE
:10546A00F9E4342D1229631228A412297B54F0126C
:05547A0013F6021A1BED
:0344B6009014D18E
:1044B90012298F24FAFFE5F034FFFE9014D1E0D3DE
:1044C9006480948090126F75F003EF400A122854AB
:1044D900A3E475F0048009122854A374FF75F0FC55
:1044E9001214C790126F122850121807902DDD125E
:1044F900294B400C122A2490126F122850121827A7
:1045090090126F122850121807C3902DD512294CFA
:10451900500C12291990126F122850121827901254
:104529006F12285012293E1213A71228EAC333CE5C
:0C45390033CED8F9122A99EDF0021A1BBB
:104FBD00EF12185C4FDD014FE7024FF1034FFB0479
:104FCD005000FC4FF6FD4FECFE4FE2FF0000500588
:104FDD007E007F01227EFF7FFF227E007F10227EDA
:104FED00FF7FF0227E007F40227EFF7FC0227E0069
:0C4FFD007FFF227EFF7F0122E4FEFF22E6
:035009009014C43C
:10500C0012288BE92FF9EA35F0FA9014C4E0FF125C
:10501C004FBD900001EE8FF0121556900001122A30
:10502C002B4008900001E4F5F08011C3EF94CFEE13
:10503C009403400B900001740375F0CF1215A3126A
:08504C001A1B9014C5122A651D
:015054002239
:034754009014338B
:1047570012288BE92FF9EA35F0FA90143512182749
:104767001228EBC333CE33CED8F92456F9740D3E55
:10477700FA7B01901438121827901433E0FF124F78
:10478700BD12293BEE8FF0121556900003122A2B0B
:10479700401312293BE4F5F01215A390143812299F
:1047A7003E7402801CC3EF94CFEE9403400B122992
:1047B7003B740375F0CF1215A390143812293E7479
:0D47C70005121408121A1B901434122A65F2
:0147D40022C2
:10430200900DA01228E17BFF90118C122868901169
:10431200A4F0900DA4E090118F1228619011A6F0E4
:10432200900DA8E09011921228619011A8F0900DC2
:10433200AC1228E19011951228689011AAF0900D04
:10434200B01228E19011981228689011ACF0E4FDA7
:10435200122974EF7802C333CE33CED8F924A1F5F3
:1043620082740D3EF583E0601024FD600C14600E33
:104372002402701912291980081229588003122A5E
:104382002412297490116E1228501218270DED6410
:034392000570BDF6
:014395002205
:104854001245CC7A2C79C91228AA9011BB1228D2FD
:104864007A12793A122A389011BE1229027A1279F0
:104874004D90138B122875121A867A2C79DC122823
:10488400AA9011C11228D27A127960122A38901192
:10489400C41229027B017A12796390138B121827B0
:1048A4009011C71229BD7A127965122A70121A86DC
:1048B40012286E125368125CA77E2E7F017D0A12A5
:0C48C4004B497A11799B1229280257A257
:10439600E4901238F07F03124CC67F39125A581235
:1043A60043027BFF7A2C79F11228AC90116E122809
:1043B600D27A1179A4122A389011711229027B013E
:1043C6007A1179A690138B122877121A867BFF7AB8
:1043D6002D79041228AC9011741228D27A1179A87A
:1043E600122A389011771229027B017A1179AA9044
:1043F600138B12182790117A1229BD7A1179AC12F3
:104406002A70121A8612286E125368125CA77E2E24
:104416007F517D0A124B497A1179A0122928025739
:01442600A2F3
:1050A0007BFF7A2D791B1228AC901262E0FFE4128C
:1050B000296C122AA3121A867BFF7A2C79C2122835
:1050C000AC7B017A12794F121A8612286E1253683D
:1050D000125CA77E2E7F837D01124B497B017A11E2
:0850E00079A112292A0257A24E
:105238007BFF7A2D79381228AC900FB6E075F00311
:10524800A4240FF81217EE1228D87A12793C121AF1
:105258008612286E125368125CA77E2E7F8D7D0100
:0F526800124B497B017A1179A212292A0257A20F
:104AE6007BFF7A2D79551228AC900FB7122A5A906F
:104AF6001382121827900FB9E060047F5280027F5C
:104B060072901385EFF0122AA3121A867BFF7A2D74
:104B1600795F1228AC900FB8122A5A1228D87A1246
:104B2600794F121A8612286E125368125CA77E2ECF
:104B36007F977D03124B497B017A1179A312292AAB
:034B46000257A271
:1045CC00900D4C1228E17BFF90117D1228689012FF
:1045DC003AF0900D501228E1901180122868901238
:1045EC004DF0900D541228E190118312286890120E
:1045FC0060F0900D581228E19011861228689012E4
:10460C0063F0900D5C1228E19011891228689012C9
:10461C0065F0E4FD122974EF7802C333CE33CED8A3
:10462C00F9122A7BE07BFFB406067A2D79E580042B
:10463C007A2D79E11229749011BB12285012182787
:05464C000DEDB405CFE7
:014651002246
:1056D10090119D121807EB8A8389827BFF7A2E79BC
:1056E100A6F4700A74A665827004742E6583700333
:0456F100125C4F22D6
:104BAB00E49014C6F09014C6E0FFC364809499504F
:104BBB004F901239E075F07D900DC21217E2EF3372
:104BCB0095E0FE75F005EF1217E2EE75F005A425E2
:104BDB0083F583E0540F9014C66009E025E02407A9
:104BEB00A3F08007E025E02406A3F07F03124CC658
:104BFB009014C7E0FF125A589014C6E004F080A539
:014C0B002286
:102EA600901238E0600D7F03124CC67F38125A58D4
:102EB600124BAB90130BE0FFC39419400BEFD39466
:102EC600265005EF24F2800490130BE0901451F085
:102ED600901451E0FF1219DA500890116DE0901429
:102EE60051F0901451E0FF642C6004EFB42908906F
:102EF600116DE0901451F0901451E0FF90116DF0B7
:102F06001228A475F005EFA4F58285F0831213A7A5
:102F1600540F901451600CE024BC12295FC3E9944D
:102F2600BC800A1228E1122964C3E994A3901450C4
:102F3600F0901450E012289FE92F122981C4540FF3
:102F4600901452F090000112151EFF901453E5F0F4
:102F5600F0A3EFF090000312151EFF901455E5F054
:102F6600F0A312298F24FA1228EAC333CE33CED81F
:102F7600F9122A99E024FE600A14600C14600E24EB
:102F860004701612291980081229588003122A245F
:102F960090126F12284A12182790127B1228FC9062
:102FA60011B9F07BFF7A2D79641228AC122991FFB2
:102FB600E5F012296C901238E07BFF60067A2D79D5
:102FC6007780047A2D797A9013841218277B017AF8
:102FD6001179B9901387121827ED1229CC12180708
:102FE60012183C90138A121827122AA3121A861254
:102FF60028EBC333CE33CED8F92459F582740D3E6F
:10300600F583E07BFFB4051B7A2D797D1228AC127F
:1030160029AD901455E0FFA3E0901384CFF0A3EF01
:10302600F080127A2D798E1228AC1229AD7A2D797C
:103036009FA31218277B017A12794F121A86C39022
:103046001340E0941090133FE09427400D12286E31
:10305600125368E490133FF0A3F0125CA77E2E7F14
:10306600337D06124B497B017A11799C12292A027B
:0230760057A25F
:03000000020C00EF
:03000300021A03DB
:03000B00021A06D0
:03001300021A09C5
:03001B00021A0CBA
:03002300021A0FAF
:03002B00021A12A4
:03003300021A1599
:03003B00021A188E
:03004300021A1B83
:03004B00021A1E78
:03005300021A216D
:03005B00021A2462
:03006300021A2757
:03006B00021A2A4C
:03007300021A2D41
:03007B00021A3036
:03008300021A332B
:03008B00021A3620
:03009300021A3915
:03009B00021A3C0A
:0300A300021A3FFF
:100C0000787FE4F6D8FD9000007F007E20E4F0A31A
:0A0C1000DFFCDEFA75817E020C5550
:100C1A00020C9AE493A3F8E493A34003F68001F24A
:100C2A0008DFF48029E493A3F85407240CC8C333DB
:100C3A00C4540F4420C8834004F456800146F6DFAA
:100C4A00E4800B0102040810204080904A1EE47ED2
:100C5A00019360BCA3FF543F30E509541FFEE4939F
:100C6A00A360010ECF54C025E060A840B8E493A366
:100C7A00FAE493A3F8E493A3C8C582C8CAC583CA91
:100C8A00F0A3C8C582C8CAC583CADFE9DEE780BE49
:014A81000034
:10138E00BB010689828A83E0225002E722BBFE025D
:09139E00E32289828A83E4932290
:1013A700BB010CE58229F582E5833AF583E02250FB
:1013B70006E92582F8E622BBFE06E92582F8E22245
:0D13C700E58229F582E5833AF583E493225F
:1013D400BB010989828A83F8E028F022500327F7A9
:1013E40022BBFE05F8E328F3228A838982F8E4937A
:0213F4002822AD
:1013F600BB010689828A83F0225002F722BBFE01D6
:02140600F322CF
:10140800F8BB010DE58229F582E5833AF583E8F01A
:10141800225006E92582C8F622BBFE05E92582C8C6
:02142800F222AE
:10142A00EF8DF0A4A8F0CF8CF0A428CE8DF0A42ED6
:02143A00FE2290
:10143C00BC000BBE0029EF8DF084FFADF022E4CC94
:10144C00F875F008EF2FFFEE33FEEC33FCEE9DEC5D
:10145C00984005FCEE9DFE0FD5F0E9E4CEFD22EDA3
:10146C00F8F5F0EE8420D21CFEADF075F008EF2FED
:10147C00FFED33FD4007985006D5F0F222C398FDDE
:05148C000FD5F0EA227B
:10149100C2D5EC30E709B2D5E4C39DFDE49CFCEE76
:1014A10030E715B2D5E4C39FFFE49EFE12143CC39E
:1014B100E49DFDE49CFC800312143C30D507C3E499
:0614C1009FFFE49EFE22E5
:1014C700C5F0F8A3E028F0C5F0F8E58215827002B0
:0614D7001583E038F0224D
:1014DD00A3F8E0C5F025F0F0E582158270021583C2
:0614ED00E0C838F0E8221F
:1014F300BB010A89828A83E0F5F0A3E022500687C4
:10150300F009E71922BBFE07E3F5F009E319228985
:0B151300828A83E493F5F074019322B8
:10151E00BB0110E58229F582E5833AF583E0F5F00B
:10152E00A3E0225009E92582F886F008E622BBFEE8
:10153E000AE92582F8E2F5F008E222E5832AF5832E
:08154E00E993F5F0A3E99322F3
:10155600BB010DC58229C582C5833AC5830214C75E
:101566005011C58229F808E5F026F618F5F0E5824F
:1015760036F622BBFE11C58229F808E225F0F5F001
:10158600F218E23582F222F8E58229F582E5832A0D
:0D159600F58374019325F0F5F0E4933822FD
:1015A300F8BB0111E58229F582E5833AF583E8F07A
:1015B300E5F0A3F0225009E92582C8F608A6F02237
:0D15C300BBFE09E92582C8F2E5F008F2221E
:0D15D000EF2BFFEE3AFEED39FDEC38FC226A
:1015DD00E88FF0A4CC8BF0A42CFCE98EF0A42CFCAD
:1015ED008AF0EDA42CFCEA8EF0A4CDA8F08BF0A42B
:1015FD002DCC3825F0FDE98FF0A42CCD35F0FCEB8A
:10160D008EF0A4FEA9F0EB8FF0A4CFC5F02ECD394E
:0F161D00FEE43CFCEAA42DCE35F0FDE43CFC22BB
:10162C0075F008758200EF2FFFEE33FECD33CDCC75
:10163C0033CCC58233C5829BED9AEC99E5829840F8
:10164C000CF582EE9BFEED9AFDEC99FC0FD5F0D6D5
:10165C00E4CEFBE4CDFAE4CCF9A88222B800C1B9FF
:10166C000059BA002DEC8BF084CFCECDFCE5F0CB3D
:10167C00F97818EF2FFFEE33FEED33FDEC33FCEB76
:10168C0033FB10D703994004EB99FB0FD8E5E4F931
:10169C00FA227818EF2FFFEE33FEED33FDEC33FC1E
:1016AC00C933C910D7059BE99A4007EC9BFCE99A12
:1016BC00F90FD8E0E4C9FAE4CCFB2275F010EF2F57
:1016CC00FFEE33FEED33FDCC33CCC833C810D70757
:1016DC009BEC9AE899400AED9BFDEC9AFCE899F892
:0E16EC000FD5F0DAE4CDFBE4CCFAE4C8F92225
:10517000C2D5E830E70FB2D5E4C39BFBE49AFAE46A
:1051800099F9E498F8EC30E717B2D51251A6121647
:1051900068E4C39BFBE49AFAE499F9E498F8800385
:1051A00012166830D50DE4C39FFFE49EFEE49DFD1A
:0451B000E49CFC225D
:1016FA00EB9FF5F0EA9E42F0E99D42F0EC6480C867
:06170A0064809845F02206
:10171000EB9FF5F0EA9E42F0E99D42F0E89C45F02F
:0117200022A6
:10172100E8600FECC313FCED13FDEE13FEEF13FFA6
:03173100D8F122CA
:10173400E8600FEFC333FFEE33FEED33FDEC33FC13
:03174400D8F122B7
:0C174700E0FCA3E0FDA3E0FEA3E0FF2215
:0C175300E0F8A3E0F9A3E0FAA3E0FB2219
:10175F007401FF3395E0FEFDFCA3A3A3E0CF2FF0B0
:10176F00E582158270021583E0CE3EF0E582158288
:10177F0070021583E0CD3DF0E5821582700215836E
:05178F00E0CC3CF0225B
:0C179400ECF0A3EDF0A3EEF0A3EFF022C8
:1017A000A8828583F0D083D0821217B71217B712A0
:1017B00017B71217B7E473E493A3C583C5F0C583C5
:1017C000C8C582C8F0A3C583C5F0C583C8C582C893
:0117D00022F6
:1017D100F5F0C582A4C582C5F0C583A42583F58330
:0117E10022E5
:0C17E200A42582F582E5F03583F5832212
:0917EE00E6FB08E6FA08E6F92220
:1017F700FAE6FB0808E6F925F0F618E6CA3AF622F3
:09180700E0FBA3E0FAA3E0F922E2
:10181000F8E0FBA3A3E0F925F0F0E5821582700261
:071820001583E0FA38F02205
:09182700EBF0A3EAF0A3E9F022C2
:0C183000E493FB740193FA740293F92214
:10183C00BB010789828A830218075005E9F8021751
:10184C00EEBBFE05E9F802188889828A83021830FB
:10185C00D083D082F8E4937012740193700DA3A31B
:10186C0093F8740193F5828883E47374029368602F
:06187C00EFA3A3A380DF2F
:061882008A838982E473F1
:101A2100E578247FF582E43413F583E0057822908C
:101A3100137C30070390137FE475F0011218100234
:101A4100138E2000E97F2ED2008018EF540F2490CE
:101A5100D43440D4FF30040BEF24BFB41A00500338
:101A61002461FFE57960021579057CE57C7002054A
:101A71007B30070E90137CE475F001121810EF0211
:101A810013F60256857403D2078003E4C207F57882
:101A910090137C121827E4F579F57BF57CE57960E4
:101AA100077F20121A6480F5757AFFC201C200C255
:101AB10002C203C205C206C208121A30FF700D30FD
:101AC10007057F00121A75AF7CAE7B22B4255FC279
:101AD100D5C204121A30FF24D0B40A00501A75F08E
:101AE1000A787930D50508B6FF0106C6A426F62086
:101AF100D5047002D20380D924CFB41A00EF500468
:101B0100C2E5D204021C76D20180C6D20080C0D2C6
:101B11000280BCD2D580BAD20580B47F20121A646B
:101B21002002077401B5790040F1121A21FF121A3F
:101B310064021A9ED208D2068095121A21FB121A4B
:101B410021FA121A21F94A4B700679477A1D7BFF57
:101B510020022EE579602A7E008E827583001213A1
:101B6100A760060EEE657A70F0C2D5EBC0E0EAC060
:101B7100E0E9C0E0EE121CBDD0E0F9D0E0FAD0E01F
:101B8100FB12138EFF60AAEBC0E0EAC0E0E9C0E0FF
:101B9100121A64D0E02401F9D0E03400FAD0E0FB5D
:101BA100E57A0460DCD57AD980877BFF7A1C79B924
:101BB100D202809C791080027908C206C20880088E
:101BC100D2D5790A8004790AC2D5E57A047002F582
:101BD1007AE4FAFDFEFF121A21FC7B0820011312A0
:101BE1001A21FD7B1030000A121A21FE121A21FF60
:101BF1007B20EC3382D592D55013C3E43000069F8D
:101C0100FFE49EFEE42001039DFDE49CFCE4CBF88F
:101C1100C201EC700CCFCECDCCE824F8F870F38083
:101C210017C3EF33FFEE33FEED33FDEC33FCEB3343
:101C3100FB994002FB0FD8E9EB300105F8D0E0C475
:101C410048B201C0E00AEC4D4E4F78207B0070C2D3
:101C5100EAB57A0040BCC0E0121CBFD0F0D0E02051
:101C61000104C4C0E0C4B201C0F0121A4DD0F0D5D5
:101C7100F0EB021A9E12185C1B3B531BB5581B0C50
:101C81004C1B08421BB94F1BC1441BC1491B2143BB
:081C91001BC7551BAB461BAB42
:101C9900451BAB471D67501B102D1B142E1B372BE3
:101CA9001B18231B35201D502A1AD04800001B2F52
:101CB9003F3F3F00790AA2D5200314300509B91026
:101CC900020404B9080104A2D52006025001042027
:101CD90002689202B579005034C0E07F20300319C0
:101CE9007F30A20272067205500F121D16C202C27F
:101CF90006C205C2087F30800F300503E9C0E01233
:101D09001A64300503D0E0F9D0E0B579CC30051775
:101D19007F30B9100C121A647F583004077F78801D
:101D290003B90803121A643002057F2D021A647F71
:101D3900202008F87F2B2006F322920280CF286EFC
:101D4900756C6C2900D201121A213001F8C2017890
:101D59007930D50108F6021AD02D50434958121A84
:101D6900212403B405004001E4901D6293121A5521
:0D1D7900743A121A55D203757904021BB595
:09188800E2FB08E2FA08E2F92291
:10568500EFB40A07740D125690740A309811A89950
:10569500B8130CC2983098FDA899C298B811F63085
:0756A50099FDC299F599225D
:00000001FF
